:100000000C9465040C9482040C9482040C94820475
:100010000C9482040C9482040C9482040C947C0949
:100020000C9482040C9482040C945E0C0C94820454
:100030000C9482040C9412080C9441080C948204D1
:100040000C9482040C9482040C9482040C94820418
:100050000C9482047B067D068406CA06FD06FD0616
:10006000FD06FD06FD06FD06FD06FD06FD06FD0678
:10007000FD067905FD06F7057705FA05AD05780655
:10008000B505C5057905F106FD06FD06FD06CD059C
:10009000000727066006EC05F105C805F4051906FA
:1000A000CB054D0655066306FD06FD06FD06FD065D
:1000B000FD06FD06FD06F705FD06FA05AD05780609
:1000C000B505C5057905F106FD06FD06FD06CD055C
:1000D000000727066006EC05F105C805F4051906BA
:1000E000CB054D0655066306004080C0105090D0E9
:1000F0002060A0E03070B0F0044484C4145494D460
:100100002464A4E43474B4F4084888C8185898D80F
:100110002868A8E83878B8F80C4C8CCC1C5C9CDCBF
:100120002C6CACEC3C7CBCFC014181C1115191D1E7
:100130002161A1E13171B1F1054585C5155595D50F
:100140002565A5E53575B5F5094989C9195999D9BF
:100150002969A9E93979B9F90D4D8DCD1D5D9DDD6F
:100160002D6DADED3D7DBDFD024282C2125292D297
:100170002262A2E23272B2F2064686C6165696D6BF
:100180002666A6E63676B6F60A4A8ACA1A5A9ADA6F
:100190002A6AAAEA3A7ABAFA0E4E8ECE1E5E9EDE1F
:1001A0002E6EAEEE3E7EBEFE034383C3135393D347
:1001B0002363A3E33373B3F3074787C7175797D76F
:1001C0002767A7E73777B7F70B4B8BCB1B5B9BDB1F
:1001D0002B6BABEB3B7BBBFB0F4F8FCF1F5F9FDFCF
:1001E0002F6FAFEF3F7FBFFF76322E350A0053658A
:1001F0006C662D54657374204572726F723A2030AC
:100200006200496E697469616C697A6564210A00EB
:10021000203D3E204E6F20616E73776572206672BE
:100220006F6D20417564696F210A00203D3E204EAC
:100230006F20616E737765722066726F6D204D65F9
:100240006D6F7279210A00203D3E2043616E277454
:1002500020777269746520746F204D656D6F7279B7
:10026000210A00286429656C6574652C202867299B
:10027000657420616E696D732C2028732965742064
:10028000616E696D732C20287629657273696F6EB3
:100290000A00287429696D652C2028612975646914
:1002A0006F2C202863296F756E742C2028782943C1
:1002B0007573746F6D20636F756E740A00287929E9
:1002C0005365742061206672616D652C2073696DC1
:1002D0002870296C6520616E696D0A007428652993
:1002E00073742C20286D296F64652C20642875296F
:1002F0006D700A00506C61792053286E29616B651E
:100300000A00416C6C204C454473204F66662F4FA9
:100310006E2028302F31290A002832293A205465CE
:10032000737420416E696D2E20310A002833293AFA
:1003300020466F6E7420546573740A005379737489
:10034000656D2054696D653A2000204672616D65C7
:10035000732073746F7265640A004E657720616E56
:10036000696D6174696F6E20636F756E743A2000F9
:10037000647572617469286F296E0A004672616D36
:100380006520746F206368616E67653A200053656D
:100390006C662D546573743A203062004B696C6C46
:1003A000656420416E696D6174696F6E20436F757D
:1003B0006E746572210A00436F756C64206E6F74F1
:1003C0002061636365737320646576696365210AE0
:1003D00000417564696F20446174613A0A00436F9B
:1003E0006E74726F6C733A20572041205320442062
:1003F0005120452C207820746F20717569740A0093
:1004000052616E206F7574206F662048656170219F
:100410000A00416E696D6174696F6E2061626F726E
:10042000746564210A002869296E7465727275709A
:100430007420636F756E742C20287229616E646F4E
:100440006D2C2028712972657365740A0020496E2D
:100450007465727275707473206166746572203190
:100460003030306D7365630A00204672616D6573CC
:1004700020706572205365636F6E640A004D656D70
:100480006F72792064656C65746564210A00526539
:1004900073657420696E203530306D732E2042797B
:1004A00065210A00456E746572206672616D652073
:1004B000746F2064756D703A2000466F726D6174C0
:1004C00074696E67206D656D6F72792E2E2E200017
:1004D000446F6E65210A002866296F726D61742071
:1004E0006D656D6F72792C2028772972697465208B
:1004F000746578740A004475726174696F6E3A208D
:100500000053746172743A200038204C617965722E
:1005100062797465732E2E2E0A0053746F72696EA1
:100520006720696E2038206672616D65732E2E2EED
:100530000A00456E64653A200043756265206D6F60
:10054000646520656E7465726564210A0041756496
:10055000696F206D6F646520656E746572656421D6
:100560000A00546578743A2000E801EE0102021096
:10057000022B02470263029202BD02DC02F4020275
:100580000319032C033C034A035A0370037C038EB4
:10059000039C03B703D103DE030004120426044DB9
:1005A0000469047D048E04A404BA04D004D704F6BC
:1005B00004010509051A05320539054D0562055383
:1005C0007472696E67206E6F7420666F756E642139
:1005D0000A0000000000000000000C1E1E0C0C00B1
:1005E0000C00363636000000000036367F367F3687
:1005F00036000C3E031E301F0C00006333180C66DF
:1006000063001C361C6E3B336E00060603000000C0
:100610000000180C0606060C1800060C1818180C1A
:10062000060000663CFF3C660000000C0C3F0C0C12
:10063000000000000000000E0C060000003F00005B
:10064000000000000000000C0C006030180C0603D5
:1006500001001E333B3F37331E000C0F0C0C0C0CFB
:100660003F001E33301C06333F001E33301C303336
:100670001E00383C36337F3030003F031F303033AC
:100680001E001C06031F33331E003F3330180C06B8
:1006900006001E33331E33331E001E33333E301824
:1006A0000E0000000C0C000C0C0000000C0C000EE6
:1006B0000C06180C0603060C180000003F003F0053
:1006C0000000060C1830180C06001E3330180C0001
:1006D0000C003E637B7B7B031E000C1E33333F33D9
:1006E00033003F66663E66663F003C660303036672
:1006F0003C003F36666666363F007F46161E16464D
:100700007F007F46161E16060F003C6603037366C5
:100710007C003333333F333333001E0C0C0C0C0C92
:100720001E007830303033331E006766361E366662
:1007300067000F06060646667F0063777F6B63637C
:10074000630063676F7B736363001C3663636336A8
:100750001C003F66663E06060F001E3333333B1E09
:1007600038003F66663E1E3667001E33071C38336E
:100770001E003F2D0C0C0C0C1E003333333333336F
:100780003F0033333333331E0C006363636B7F7777
:1007900063006363361C366363003333331E0C0C13
:1007A0001E007F33190C46637F001E0606060606F0
:1007B0001E0003060C18306040001E181818181888
:1007C0001E00081C3663000000000000000000004E
:1007D00000FF0C0C18000000000000001E303E332B
:1007E0006E0007063E6666663D0000001E3303335A
:1007F0001E003830303E33336E0000001E333F039E
:100800001E001C36060F06060F0000006E33333E36
:10081000301F0706366E666667000C000E0C0C0C67
:100820001E0018001E1818181B0E070666361E3606
:1008300067000E0C0C0C0C0C1E000000377F6B6365
:10084000630000001F333333330000001E333333A3
:100850001E0000003B66663E060F00006E33333E0E
:10086000307800001B3636060F0000003E031E30B5
:100870001F00080C3E0C0C2C1800000033333333DF
:100880006E0000003333331E0C00000063636B7F87
:100890003600000063361C36630000003333333EFD
:1008A000301F00003F190C263F00380C0C070C0CC1
:1008B00038001818180018181800070C0C380C0C01
:1008C00007006E3B00000000000011241FBECFE5B2
:1008D000D8E0DEBFCDBF11E0A0E6B0E0ECE0F9E586
:1008E00002C005900D92AA3DB107D9F712E0AAED1A
:1008F000B1E001C01D92A13EB107E1F70E940907D6
:100900000C94842C0C9400008FEF8ABB8CEF81BB7D
:1009100098E197BB84BB87B3866087BBB8980E9479
:100920008D0A89E190E068E040E021E00E948408BF
:100930000E94D20A0E94550C789485E690E00E94AD
:100940002C0A0895CF93DF930E94370CC1E00097E3
:1009500009F0C0E060E070E0CB0141E00E94700B64
:10096000009711F4C26002C00E94F72980E063E2A0
:100970000E94530D80E00E94610D833211F0C4602B
:1009800002C0CC2341F181E00E94700D0E945A09FF
:10099000DC2F8C2F90E062E872E042E050E00E9491
:1009A000012C0E945A098AE00E941A09C0FF05C062
:1009B00083E00E94700D0E945A09D1FF05C084E0B7
:1009C0000E94700D0E945A09D2FF05C085E00E9466
:1009D000700D0E945A098C2FDF91CF910895AF922C
:1009E000BF92CF92DF92EF92FF920F931F93CF931C
:1009F000DF9380E490E00E945D29C82FD92F2097D3
:100A000031F488E10E94700D0E945A094EC0E82F0F
:100A1000F92FCF01805C9F4F1192E817F907E1F79A
:100A200000E010E191E0C92ED12CA895CE010E94E2
:100A30002C0A0E94890A8823E1F30E94D42A5C01CF
:100A40000E94D42A7C010E94D42A9C01C701B801CB
:100A50000E94D228E62FF0E083E0EE0FFF1F8A9578
:100A6000E1F7C501B8010E94D228E60FF11DEC0F95
:100A7000FD1FC901B8010E94D228C60102C0880F1B
:100A8000991F6A95E2F7BC018081862780830E94C6
:100A9000B608882351F289E10E94700D0E945A091C
:100AA000CE010E94F7290E94C408DF91CF911F91C7
:100AB0000F91FF90EF90DF90CF90BF90AF9008958F
:100AC000CF92DF92EF92FF920F931F93CF93DF931A
:100AD00090E0C0978A34910508F08FC1865D9F4FE2
:100AE000FC01EE0FFF1F0590F491E02D099482E4C4
:100AF00085C186E00E94700D0E945A0987E00E941D
:100B0000700D0E945A0988E00E94700D0E945A09D7
:100B100089E00E94700D0E945A098AE00E94700DBF
:100B20000E945A098AE10E94700D0E945A0982E2CD
:100B30000E94700D0E945A0981E10E94700D0E946E
:100B40005A098BE00E94700D0E945A098CE00E94A5
:100B5000700D0E945A098DE018C180E090E00E945B
:100B6000420D82E40E941A090CC080E20E94700DBE
:100B70000E945A090E94060D81E20E94700D0E9497
:100B80005A0981E08093DB013BC10E945C1938C1A6
:100B90000E940D14F6CF80E0F8C04091DC01242FB4
:100BA00030E08091A50090E001972817390724F4E0
:100BB0004F5F4093DC0102C01092DC018091DC01A8
:100BC000882341F06AE00E94EA1A80E20E941A0932
:100BD00089E2DBC088E2D9C081E08093DA018EE14E
:100BE000D4C00E94EF040CC10E94911909C10E9457
:100BF000601906C10E94260D62E872E04AE050E0EA
:100C00000E94012C0E945A0980E690E00E945A0935
:100C10008091DB0190E062E872E04AE050E00E94DF
:100C2000012C0E945A0983E690E00E945A098FE045
:100C3000ACC08FE10E94700D0E945A098AE00E94A8
:100C4000D71A0E94D40CEC010E944B1A4DC084E2CA
:100C50000E94700D0E945A098AE00E94D71AC82F7C
:100C600087E20E94700D0E945A098AE00E94D71AFA
:100C7000E82E83E20E94700D0E945A098AE00E94C9
:100C8000D71A082F06C08C2F90E0602F0E94F50C19
:100C9000CF5FEC16C0F781E278C08AE20E94700D47
:100CA0000E945A090E94901BABC080E10E94700D07
:100CB0000E945A098AE00E94D71A0E94420D61CF11
:100CC0000E943C1B9DC082E10E94700D0E945A0947
:100CD0008AE00E94D71A082F0E94FA1AEC01802F8E
:100CE00090E0BE010E94E40CCE010E94F72988C06A
:100CF0000E94A20485C080E001C08FEF0E94610ABB
:100D000081E08093DF017CC085E690E00E94870D42
:100D1000DD2441E0E42EF12C29C0188200E010E02F
:100D2000C701002E02C0880F991F0A94E2F728819C
:100D3000282B288385E690E00E942C0A05C0A89500
:100D40000E94B6088823F1F40E94890A8823B9F327
:100D50000F5F1F4F0830110519F7CA942196CC2058
:100D6000E1F6D394FD2DF83008F0DD24CD2DD0E050
:100D700033E0CC0FDD1F3A95E1F7CB59DF4F28E088
:100D8000C22ECBCF0E94C40889E10E94700D0E9440
:100D90005A0936C085E690E00E94870DC0E28C2F8C
:100DA0000E943D1CCE3710F4CF5F01C0C0E2282F57
:100DB000392FD901E5E6F0E08D91819380E0ED36A1
:100DC000F807D1F7CF0108970E942C0A05C0A89513
:100DD0000E94B6088823B1F60E94890A8C30F8F682
:100DE000F6CF0E94210A42E852E02AE030E00E9459
:100DF000222C0E945A098AE001C083E20E941A094B
:100E0000DF91CF911F910F91FF90EF90DF90CF90E6
:100E100008959F92AF92BF92CF92DF92EF92FF928E
:100E20000F931F93CF93DF9314BE88E10FB6F8940E
:100E300081BD11BC0FBE0E9484042EE088E190E0C9
:100E40000FB6F894A89581BD0FBE21BD0E94A204E3
:100E500090E080FF03C021E02093DD018670907058
:100E6000009719F081E08093DE0180E00E94700D10
:100E70000E945A098091DE01882331F40E94260DD8
:100E80008C011092DC0105C081E08093DC0100E060
:100E900010E08091DD01882321F40E94ED0D8F5F29
:100EA00003C01092DC0181E08093A5000E947712BC
:100EB000C82E82E00E94700D0E945A099924BB241A
:100EC000C0E0D0E0AA24A394DD240894C108D1088E
:100ED0008091DA01882309F4A8958091DB018823A9
:100EE00049F01092DB018091DE01882319F40E9401
:100EF000260D8C010E94B608882321F00E94C408A8
:100F00000E9460058091E001882371F080E0B09B31
:100F10002AC0E7E8F1E03197F1F700C00000815006
:100F2000B1F71092E0011FC080E0B0991CC0E7E863
:100F3000F1E03197F1F700C000008150B1F7A092C5
:100F4000E0014091DC01842F90E02091A50030E089
:100F5000215030408217930724F44F5F4093DC0107
:100F600002C01092DC018091DC018823E1F58091C0
:100F7000DF01882309F0ACCF0115110511F1809133
:100F8000DE018823F1F40E94890A981608F0A0CFA8
:100F9000C8010197C817D90710F4219602C0C0E014
:100FA000D0E0CE010E94D40C7C01009789F1FC01B5
:100FB000E05CFF4F90800E942C0AC7010E94F72935
:100FC00087CF0E94890A981608F082CF2B2D30E037
:100FD0002C153D0514F4B39401C0BB248B2D0E9445
:100FE000F513982E75CF8091DD018823C1F40E94FE
:100FF000890A882309F46CCF0E94370C009731F0DE
:101000006091DC0161500E943E0E62CF1092DC01C3
:1010100085E690E00E942C0A58E1952E59CF109257
:10102000DC0156CF1F920F920FB60F9211248F93AF
:101030009F93EF93FF93E091E301F091E4018CB172
:10104000E550FE4F80838091E3019091E4018F3160
:10105000910550F48091E3019091E4010196909301
:10106000E4018093E30104C01092E4011092E301D3
:10107000FF91EF919F918F910F900FBE0F901F9056
:1010800018951F920F920FB60F9211242F933F9332
:101090008F939F93EF93FF932091E5013091E601A9
:1010A0008091E7019091E80128173907F1F0E0916C
:1010B000E501F091E601E55EFD4F80818CB98091FC
:1010C000E5019091E6018F31910550F48091E501A1
:1010D0009091E60101969093E6018093E50109C0A5
:1010E0001092E6011092E50104C081E08093A60011
:1010F0005598FF91EF919F918F913F912F910F9074
:101100000FBE0F901F901895433060F5362F355065
:10111000343040F5322F3150323030F5442341F035
:1011200030B5306230BD423019F430B5306130BD79
:10113000223019F420B5286020BD653061F066309A
:1011400011F0683029F420B5226020BD663019F016
:1011500020B5246020BD90BD89B98AB188698AB95B
:1011600080E0089581E0089581E008954091E101D3
:101170005091E2012091E3013091E40181E04217B6
:10118000530709F480E008952091E1013091E201D4
:101190008091E3019091E4012817390729F1E0914A
:1011A000E101F091E201E550FE4F8081E091E10123
:1011B000F091E201E550FE4F10822091E101309163
:1011C000E2012F31310558F42091E1013091E20123
:1011D0002F5F3F4F3093E2012093E1010895109279
:1011E000E2011092E101089580E008958091E70105
:1011F0009091E8012091E5013091E6010196821776
:10120000930791F08091E5019091E601009779F4C0
:101210002091E7013091E80181E090E02F31310524
:1012200041F080E090E0089581E090E0089580E052
:1012300090E008952091E7013091E8014091E501A7
:101240005091E6012F5F3F4F2417350799F3209106
:10125000E5013091E6012115310539F42091E701CE
:101260003091E8012F31310529F3E091E701F09148
:10127000E801E55EFD4F80838091E7019091E801F0
:101280008F31910550F48091E7019091E80101962A
:101290009093E8018093E70104C01092E801109256
:1012A000E7018091A600813021F41092A600559AA2
:1012B0005D9A0895CF93DF93C82FD92F02C00E9463
:1012C0001A0989918823D9F7DF91CF9108951AB827
:1012D00010BC10BC19B81092E2011092E1011092FA
:1012E000E6011092E5011092E4011092E3011092E0
:1012F000E8011092E70108951F920F920FB60F9226
:1013000011242F933F934F935F936F938F939F93EA
:10131000AF93BF93EF93FF938091EC018091E9012C
:10132000882321F01092EB011092E90112BA88B3E0
:10133000877E88BB80E090E021E030E045B34370D9
:1013400045BB48B3497F48BBE091EB01F0E043E087
:10135000EE0FFF1F4A95E1F7E80FF91FE55CFD4F1F
:1013600040814BBB823058F065B3A901082E02C002
:10137000440F551F0A94E2F7642B65BB0CC068B399
:10138000AC014F5F5F4FF90102C0EE0FFF1F4A959E
:10139000E2F76E2B68BB01968830910579F62091B3
:1013A000EB0181E090E0AC0102C0440F551F2A958B
:1013B000E2F742BB28B33091EB0102C0880F991FBE
:1013C0003A95E2F733E0880F991F3A95E1F7887173
:1013D000277E822B88BB8091EB01873030F480918F
:1013E000EB018F5F8093EB0107C01092EB018091BE
:1013F000EA018F5F8093EA011092EC018091ED0188
:101400009091EE01A091EF01B091F0010196A11D24
:10141000B11D8093ED019093EE01A093EF01B09385
:10142000F001FF91EF91BF91AF919F918F916F91DB
:101430005F914F913F912F910F900FBE0F901F9092
:1014400018952091ED013091EE014091EF015091FE
:10145000F001B901CA010895CF93DF936FB7F894F3
:1014600021E02093E9011092EA011092EC01482F4B
:10147000592F87E090E01DC0ED91F0E0E851FF4F5B
:10148000E491E095E90173E0CC0FDD1F7A95E1F777
:10149000C80FD91FC55CDD4FE8832F5F3F4F283051
:1014A000310551F7485F5F4F01972FEF8F3F92074C
:1014B00021F0DA0120E030E0DFCF6FBFDF91CF9184
:1014C00008959FB7F89421E02093E9011092EA0172
:1014D0001092EC0120E030E0809510C0FB01E40F99
:1014E000F51FE55CFD4F80834F5F5F4F483051052E
:1014F000A9F72F5F3F4F2830310549F040E050E019
:10150000B901E3E0660F771FEA95E1F7E7CF9FBFE8
:1015100008958091EA01869508958EB589608EBD03
:1015200082EC92EA9BBD8ABD80E189BF80E00E9487
:10153000610A789480E090E061E01DC07FB7F89484
:10154000FA01E20FF31FE55CFD4FA081108260936A
:10155000E9011092EA011092EC017FBF7091EA015B
:101560007723E1F32F5F3F4F2830310539F701969C
:101570008830910549F020E030E0AC01F3E0440F01
:10158000551FFA95E1F7DACFF8941092ED01109219
:10159000EE011092EF011092F0011092EA01109208
:1015A000EC01089511B88CE080B9089594EA96BFD3
:1015B00006B607FEFDCF91B1987F983011F09031BB
:1015C00079F483B984E886BF06B607FEFDCF91B1F2
:1015D000987F983139F081E0903429F480E00895C3
:1015E00081E0089580E0089544EA34E824E946BFA4
:1015F00006B607FEFDCF91B1987F983011F090317B
:10160000B1F783B936BF06B607FEFDCF91B1987F1B
:10161000903211F0983529F426BF06B604FCFDCFB0
:10162000E6CF08950E94D60A089584E986BF06B6DB
:1016300004FCFDCF089583B984E886BF06B607FE93
:10164000FDCF91B1987F81E0983209F480E0089550
:1016500084EC86BF06B607FEFDCF83B1089584E80B
:1016600086BF06B607FEFDCF83B10895DF92EF92E5
:10167000FF920F931F93DF93CF930F92CDB7DEB7F7
:101680007B018C0180E0E81680E0F80681E0080725
:1016900080E0180718F490EAD92E02C082EAD82E0A
:1016A0008D2D0E94D60A882389F48F2D0E941B0B52
:1016B0008E2D0E941B0B8D2D81600E94120B0E94AB
:1016C0002F0B89830E94150B898101C080E00F9048
:1016D000CF91DF911F910F91FF90EF90DF900895D0
:1016E0008F929F92AF92BF92CF92DF92EF92FF9232
:1016F0000F931F93CF93DF934B015C0180E088161B
:1017000080E0980681E0A80680E0B80618F430EA88
:10171000E32E02C022EAE22E042F10E0C8010E944C
:101720005D29EC016C01009731F488E10E94700D95
:101730000E945A092CC08E2D0E94D60A882329F5B2
:10174000892D0E941B0B882D0E941B0B8E2D816002
:101750000E94120BBB24480108948108910807C01D
:101760000E94280BFE01EE0DFF1D8083B394EB2C2D
:10177000FF24E814F904A4F30E942F0BC00FD11F1B
:10178000219788830E94150B02C0CC24DD24C6015A
:10179000DF91CF911F910F91FF90EF90DF90CF904D
:1017A000BF90AF909F908F900895EF92FF920F930C
:1017B0001F93CF937B018C01C42F80E0E81680E05B
:1017C000F80681E0080780E0180710F480EA01C0FD
:1017D00082EA0E94D60A882359F48F2D0E941B0B9F
:1017E0008E2D0E941B0B8C2F0E941B0B0E94150B31
:1017F000CF911F910F91FF90EF900895CF92DF92BC
:10180000EF92FF920F931F93CF93DF937B018C0195
:10181000D42EC52FC22E80E0E81680E0F80681E0C5
:10182000080780E0180710F480EA01C082EA0E94ED
:10183000D60A882399F48F2D0E941B0B8E2D0E94AF
:101840001B0B8C2FCD2DD82F03C089910E941B0B11
:101850008C2F8D198C15C8F30E94150BDF91CF9139
:101860001F910F91FF90EF90DF90CF900895CF934D
:10187000DF9383E40E94D60A882389F4CBE7D2E081
:101880000E94280B899382E0C138D807C9F70E94CB
:101890002F0B809381020E94150B269702C0C0E097
:1018A000D0E0CE01DF91CF91089583B78B6083BFE5
:1018B0008AEF8CBF89B7826089BF08951F920F920B
:1018C0000FB60F9211242F933F934F935F936F9313
:1018D0007F938F939F93AF93EF93FF934091F20188
:1018E0003091F3012091F4019091F5018091F6017E
:1018F000F091F701E091F801A091F901642F6F5F79
:1019000051E0641708F050E0530F41E0531708F01E
:1019100040E0420F31E0421708F030E0390F21E09B
:10192000391708F020E0280F91E0281708F090E020
:101930009F0F81E09F1708F080E08E0F71E08E17F7
:1019400008F070E07A0F6093F2015093F301409336
:10195000F4013093F5012093F6019093F701809301
:10196000F8017093F901FF91EF91AF919F918F91E1
:101970007F916F915F914F913F912F910F900FBE8B
:101980000F901F9018952091F2013091F301409132
:10199000F4015091F5016091F6017091F701809189
:1019A000F8019091F9010895BC0126E0660F771FB8
:1019B0002A95E1F7680F791F605E7F4F80E090E025
:1019C00041E40E94700B0895AB01BC0136E0660F44
:1019D000771F3A95E1F7680F791F605E7F4F80E0CF
:1019E00090E021E40E94FE0B0895462F9C0156E0F2
:1019F000220F331F5A95E1F7280F391F205A3F4F06
:101A0000B90180E090E00E94D50B0895EF92FF921B
:101A10000F931F93EE24FF248701C801B70140E014
:101A20000E94D50BA8950894E11CF11C011D111D05
:101A300080E0E81680E0F80682E0080780E01807FA
:101A400061F71F910F91FF90EF900895CF9360E0A1
:101A500070E0CB010E94360BC82F61E070E080E09F
:101A600090E00E94360B2C2F30E0582F40E0242BC2
:101A7000352B87E0213E380710F020EE37E0C90112
:101A8000CF910895CF93482FC92F60E070E0CB012C
:101A90000E94D50B61E070E080E090E04C2F0E9446
:101AA000D50BCF910895462F8E3150F490E00296D9
:101AB0009C01B901882777FD8095982F0E94D50B4E
:101AC00008958E3158F4682F70E06E5F7F4F88273D
:101AD00077FD8095982F0E94360B089580E0089539
:101AE0008B3248F4E82FF0E0EE0FFF1FE759FA4F72
:101AF0002591349104C0EFEBF5E02591349182E813
:101B000092E0B9010E94FA2B82E892E00895282F12
:101B1000392FF90180E411928150E9F708951F935C
:101B2000CF93DF9381E490E00E945D29192FC82FA5
:101B3000D92F209731F488E10E94700D0E945A0934
:101B4000FFCFCE010E94870DFE01E05CFF4F81E0D8
:101B500080838C2F912FDF91CF911F910895A7E063
:101B6000B0E0FD01E41BF109AD01421B51099A01EE
:101B700043E0220F331F4A95E1F7E20FF31FE80F0E
:101B8000F91F81E090E002C0880F991F6A95E2F783
:101B90002081282B20830895A7E0B0E0FD01E41BFD
:101BA000F109AD01421B51099A0153E0220F331F85
:101BB0005A95E1F7E20FF31FE80FF91F81E090E07B
:101BC00002C0880F991F6A95E2F78095908198234B
:101BD000908308950E94F729089587E00895282F9B
:101BE000392FF90197E080E02191821708F4822FC4
:101BF0009150D1F70895982F662359F0E5EBF0E066
:101C000080E003C08F5F883039F021912917D0F32D
:101C100008956FE10E94B2280895282F392FF90105
:101C200027E080E090E03191830F911D2150D9F79A
:101C300067E070E00E94BE28862F08951F93CF931F
:101C4000DF93D82FC92F662321F00E940D0E823119
:101C500010F412E101C019E08D2F9C2F0E940D0E8F
:101C6000811740F49E01832F922FFC0187E011928F
:101C70008150E9F7DF91CF911F9108950F931F9342
:101C8000CF93DF93EC016730D0F4062F10E064307F
:101C900048F460E00E941E0EF801EE0FFF1FE955A8
:101CA000FF4F08C061E00E941E0EF801EE0FFF1FFB
:101CB000E955FF4F0190F081E02DCE010995DF91AC
:101CC000CF911F910F9108956F927F928F929F9263
:101CD000AF92BF92CF92DF92EF92FF920F931F933A
:101CE000CF93DF937B01142F622EC02EA82EB92E26
:101CF00001E02FE0822E912CF50181915F01662D8C
:101D00000E94FB0D782EC0E0D0E0DD2429C0013018
:101D1000C1F4CC2059F0CE01B4010E94D228262F64
:101D2000C70160E0412F0E94AF0D0DC0CE01B4018C
:101D30000E94D228462FC70160E0212F0E94AF0DDC
:101D400007C0CC2029F0C701602F412F2D2D04C0E2
:101D5000C701602F4D2D212F0E94AF0DD3942A96DD
:101D6000D714A8F20F5F083039F6DF91CF911F9199
:101D70000F91FF90EF90DF90CF90BF90AF909F902A
:101D80008F907F906F900895EF92FF920F931F9323
:101D9000CF93DF937C010E948F0DEC0110E0C7010F
:101DA000BE01412F20E000E00E94640E1F5F18304A
:101DB000B1F7CE010E942C0ACE010E94EA0DDF91FC
:101DC000CF911F910F91FF90EF900895EF92FF92A6
:101DD0000F931F93CF93DF937C010E948F0DEC0133
:101DE00010E0C701BE01412F21E000E00E94640E17
:101DF0001F5F1830B1F7CE010E942C0ACE010E945D
:101E0000EA0DDF91CF911F910F91FF90EF90089510
:101E1000EF92FF920F93CF93DF937C010E948F0D7F
:101E2000EC01C701BE0142E021E000E00E94640E27
:101E3000C70160E00E941E0EC701BE0145E020E020
:101E40000E94640ECE010E942C0ACE010E94EA0D6F
:101E5000DF91CF910F91FF90EF900895EF92FF9255
:101E60000F931F93CF93DF937C010E948F0DEC01A2
:101E700012E0C701BE01412F20E001E00E94640E84
:101E80001F5F1630B1F7CE010E942C0ACE010E94CE
:101E9000EA0DDF91CF911F910F91FF90EF90089580
:101EA0000F931F93CF93DF938C010E948F0DEC0152
:101EB000C801BE0147E020E000E00E94640ECE01B0
:101EC0000E942C0ACE010E94EA0DDF91CF911F9152
:101ED0000F9108950F931F93CF93DF938C010E946E
:101EE0008F0DEC01C801BE0147E021E000E00E9437
:101EF000640ECE010E942C0ACE010E94EA0DDF91F1
:101F0000CF911F910F910895EF92FF920F931F931E
:101F1000CF93DF93F82E062F142FE901EE2407C08C
:101F2000CE016F2D4E2D202F0E94AF0DE394E116B0
:101F3000B8F3DF91CF911F910F91FF90EF9008952B
:101F4000FF920F931F93CF93DF938C010E948F0D0D
:101F5000EC01F80180813FE1F32E6F2D0E94B22841
:101F6000482F80E060E09E010E94840FF80180818C
:101F70006F2D0E94B228482F80E061E09E010E94F0
:101F8000840FF80180816F2D0E94B228482F81E0D4
:101F900060E09E010E94840FF80181816F2D0E94F4
:101FA000B228482F80E062E09E010E94840FF80171
:101FB00081816F2D0E94B228482F80E063E09E014E
:101FC0000E94840FF80181816F2D0E94B228482F52
:101FD00081E061E09E010E94840FF80181816F2DF4
:101FE0000E94B228482F81E062E09E010E94840F87
:101FF000F80181816F2D0E94B228482F82E060E0B5
:102000009E010E94840FF80181816F2D0E94B228E9
:10201000482F82E061E09E010E94840FF8018281D6
:102020006F2D0E94B228482F80E064E09E010E943C
:10203000840FF80182816F2D0E94B228482F80E022
:1020400065E09E010E94840FF80182816F2D0E943D
:10205000B228482F81E063E09E010E94840FF801BE
:1020600082816F2D0E94B228482F81E064E09E019A
:102070000E94840FF80182816F2D0E94B228482FA0
:1020800082E062E09E010E94840FF80182816F2D40
:102090000E94B228482F82E063E09E010E94840FD4
:1020A000F80182816F2D0E94B228482F83E060E002
:1020B0009E010E94840FF80182816F2D0E94B22838
:1020C000482F83E061E09E010E94840FF801828125
:1020D0006F2D0E94B228482F83E062E09E010E948B
:1020E000840FF80182816F2D0E94B228482F84E06E
:1020F00060E09E010E94840FF80182816F2D0E9492
:10210000B228482F84E061E09E010E94840FF8010C
:1021100083816F2D0E94B228482F80E066E09E01E7
:102120000E94840FF80183816F2D0E94B228482FEE
:1021300080E067E09E010E94840FF80183816F2D8B
:102140000E94B228482F81E065E09E010E94840F22
:10215000F80183816F2D0E94B228482F81E066E04C
:102160009E010E94840FF80183816F2D0E94B22886
:10217000482F82E064E09E010E94840FF801838171
:102180006F2D0E94B228482F82E065E09E010E94D8
:10219000840FF80183816F2D0E94B228482F83E0BD
:1021A00063E09E010E94840FF80183816F2D0E94DD
:1021B000B228482F83E064E09E010E94840FF8015A
:1021C00083816F2D0E94B228482F84E062E09E0137
:1021D0000E94840FF80183816F2D0E94B228482F3E
:1021E00084E063E09E010E94840FF80183816F2DDB
:1021F0000E94B228482F85E060E09E010E94840F73
:10220000F80183816F2D0E94B228482F85E061E09C
:102210009E010E94840FF80183816F2D0E94B228D5
:10222000482F85E062E09E010E94840FF8018381BF
:102230006F2D0E94B228482F86E060E09E010E9428
:10224000840FF80183816F2D0E94B228482F86E009
:1022500061E09E010E94840FF80184816F2D0E942D
:10226000B228482F81E067E09E010E94840FF801A8
:1022700084816F2D0E94B228482F82E066E09E0183
:102280000E94840FF80184816F2D0E94B228482F8C
:1022900082E067E09E010E94840FF80184816F2D27
:1022A0000E94B228482F83E065E09E010E94840FBF
:1022B000F80184816F2D0E94B228482F83E066E0E8
:1022C0009E010E94840FF80184816F2D0E94B22824
:1022D000482F84E064E09E010E94840FF80184810D
:1022E0006F2D0E94B228482F84E065E09E010E9475
:1022F000840FF80184816F2D0E94B228482F85E059
:1023000063E09E010E94840FF80184816F2D0E947A
:10231000B228482F85E064E09E010E94840FF801F6
:1023200084816F2D0E94B228482F86E062E09E01D2
:102330000E94840FF80184816F2D0E94B228482FDB
:1023400086E063E09E010E94840FF80184816F2D76
:102350000E94B228482F87E060E09E010E94840F0F
:10236000F80184816F2D0E94B228482F87E061E038
:102370009E010E94840FF80185816F2D0E94B22872
:10238000482F83E067E09E010E94840FF801858159
:102390006F2D0E94B228482F84E066E09E010E94C3
:1023A000840FF80185816F2D0E94B228482F84E0A8
:1023B00067E09E010E94840FF80185816F2D0E94C5
:1023C000B228482F85E065E09E010E94840FF80145
:1023D00085816F2D0E94B228482F85E066E09E011E
:1023E0000E94840FF80185816F2D0E94B228482F2A
:1023F00086E064E09E010E94840FF80185816F2DC4
:102400000E94B228482F86E065E09E010E94840F5A
:10241000F80185816F2D0E94B228482F87E062E085
:102420009E010E94840FF80185816F2D0E94B228C1
:10243000482F87E063E09E010E94840FF8018581A8
:102440006F2D0E94B228482F87E064E09E010E9411
:10245000840FF80186816F2D0E94B228482F85E0F5
:1024600067E09E010E94840FF80186816F2D0E9413
:10247000B228482F86E066E09E010E94840FF80192
:1024800086816F2D0E94B228482F86E067E09E016A
:102490000E94840FF80186816F2D0E94B228482F78
:1024A00087E065E09E010E94840FF80186816F2D10
:1024B0000E94B228482F87E066E09E010E94840FA8
:1024C000F80186816F2D0E94B228482F87E067E0CF
:1024D0009E010E94840FCE010E942C0ACE010E9410
:1024E000EA0DDF91CF911F910F91FF90089580E148
:1024F00008958F929F92AF92BF92CF92DF92EF9208
:10250000FF920F931F93DF93CF9300D0CDB7DEB729
:10251000882E0E948F0D7C01B82CBB0C9924089446
:10252000811C911C880C991C00E010E0CB2CDD2450
:10253000C7FCD09424C0C701632F4A2D252F3A83AE
:1025400059830E94AF0D59815F5F3A81583099F7E6
:102550003F5F383021F405C030E0AB2CA00E50E0D6
:10256000EACFC7010E942C0A01C0A8950E94890ADF
:102570008823D9F3C7010E94870D0F5F1F4FC80141
:102580008C0D9D1D881599053CF3C7010E94F72904
:102590000F900F90CF91DF911F910F91FF90EF90CF
:1025A000DF90CF90BF90AF909F908F9008958F92C3
:1025B0009F92BF92CF92DF92EF92FF920F931F9361
:1025C000DF93CF9300D0CDB7DEB7E82E0E948F0DFA
:1025D0008C01BE2CB194BB0C23E0822E912C8E1862
:1025E0009108880C991C87E0B80EEE24FF24CB2CB0
:1025F000DD24C7FCD09424C0C801632F4B2D252FA8
:102600003A8359830E94AF0D59815F5F3A815830F8
:1026100099F73F5F383011F403C030E050E0ECCF61
:10262000C8010E942C0A01C0A8950E94890A88232B
:10263000D9F3C8010E94870DBA940894E11CF11CDB
:10264000C6018E199F09881599053CF7C8010E949B
:10265000F7290F900F90CF91DF911F910F91FF906D
:10266000EF90DF90CF90BF909F908F9008958F92C2
:102670009F92AF92BF92CF92DF92EF92FF920F9311
:102680001F93DF93CF9300D0CDB7DEB7882E0E9483
:102690008F0D7C01B82CBB0C99240894811C911CD3
:1026A000880C991C00E010E0CB2CDD24C7FCD094F2
:1026B00024C0C701652F432F2A2D3A8359830E94D6
:1026C000AF0D59815F5F3A81583099F73F5F3830DD
:1026D00021F405C030E0AB2CA00E50E0EACFC701DA
:1026E0000E942C0A01C0A8950E94890A8823D9F368
:1026F000C7010E94870D0F5F1F4FC8018C0D9D1DE4
:10270000881599053CF3C7010E94F7290F900F9097
:10271000CF91DF911F910F91FF90EF90DF90CF90BD
:10272000BF90AF909F908F9008958F929F92BF928D
:10273000CF92DF92EF92FF920F931F93DF93CF938D
:1027400000D0CDB7DEB7E82E0E948F0D8C01BE2CD5
:10275000B194BB0C53E0852E912C8E189108880CF7
:10276000991C87E0B80EEE24FF24CB2CDD24C7FC97
:10277000D09424C0C801632F452F2B2D3A83598351
:102780000E94AF0D59815F5F3A81583099F73F5FE2
:10279000383011F403C030E050E0ECCFC8010E94A3
:1027A0002C0A01C0A8950E94890A8823D9F3C80180
:1027B0000E94870DBA940894E11CF11CC6018E1981
:1027C0009F09881599053CF7C8010E94F7290F90C9
:1027D0000F90CF91DF911F910F91FF90EF90DF90BD
:1027E000CF90BF909F908F9008958031A0F4843057
:1027F00018F40E9437130FC0883020F484500E94D0
:10280000951309C08C3020F488500E94791203C0BF
:102810008C500E94D71281E008952F923F924F92E0
:102820005F926F927F928F929F92AF92BF92CF9260
:10283000DF92EF92FF920F931F93DF93CF93CDB769
:10284000DEB76C970FB6F894DEBF0FBECDBF81E444
:1028500090E00E945D29888B998B8B839C830E94DA
:10286000C30CB22EC32ED42E152F062FF72EE82E12
:10287000392E82E40E941A0974C00E94C30CA22F50
:10288000AB19F1E02A1708F0F0E0232F2C19E1E052
:10289000321708F0E0E0322F3F1BF32F31E02F1703
:1028A00008F030E0E32B342F3D1921E0431708F006
:1028B00020E0432F4E1BE42F41E03E1708F040E09C
:1028C000242B452F411B31E0541708F030E0542FE2
:1028D000521B21E0451708F020E0322B462F401B09
:1028E00021E0641708F020E0642F631B31E04617F5
:1028F00008F030E0232B472F4F1931E0741708F010
:1029000030E0742F721B21E0471708F020E0322BD3
:10291000482F4E1921E0841708F020E0842F831BF4
:1029200031E0481708F030E0232B9319921709F093
:1029300099C4882309F096C4772309F093C46623C9
:1029400009F090C4552309F08DC4EE2309F08AC420
:10295000F23008F087C4F13019F4A53F08F082C4C2
:10296000A8950E94B608882309F487CF0E94C4085E
:102970008A8B82E40E941A0984EF282EAA24A39449
:102980005524662477248824992444241F821E8297
:102990001E868B819C81805C9F4F9F8B8E8B2D82AE
:1029A000BB86CC86DD86212EB02ECF2CDE2C37C206
:1029B0000E94C30C122FAB851A1BF1E0211708F0FF
:1029C000F0E0E32FBC85EB1B21E03E1708F020E090
:1029D0003E2F3F1BF1E0E31708F0F0E02F2BA42F70
:1029E000ED85AE1BF1E04A1708F0F0E04A2F421BDC
:1029F00021E0A41708F020E0F22BA52FA21921E076
:102A00005A1708F020E05A2F5F1BF1E0A51708F0D5
:102A1000F0E02F2BA62FAB19F1E06A1708F0F0E0D9
:102A20006A2F621B21E0A61708F020E0F22B272F67
:102A30002C19A1E0721708F0A0E0722F7F1BF1E0C3
:102A4000271708F0F0E0AF2BF82FFD1921E08F17C2
:102A500008F020E08F2F8A1BA1E0F81708F0A0E013
:102A60002A2B9319921B491608F4FCC3941511F5EF
:102A7000981608F4F7C38915E9F4871608F4F2C329
:102A80007815C1F4761608F4EDC3671599F4651648
:102A900008F4E8C3561571F4541608F4E3C3451559
:102AA00049F4A31608F4DEC33A1521F4FD81F117A9
:102AB00008F4D8C3A8950E94B608882309F478CFF3
:102AC0000E94C4088B8B82E40E941A092E813F81E8
:102AD0003A8329834F864B2CBC2CCD2C8EC13D8153
:102AE0003C503A8751E04D81341708F050E08A2D70
:102AF0008F5F91E08A1508F090E0580F41E0581779
:102B000008F040E0492B450D11E0451508F010E0B4
:102B1000160D01E0161508F000E0070D81E007151D
:102B200008F080E0F82EF80C81E0F81408F080E05E
:102B3000E82EE90C81E0E91408F080E0DF84D80E8B
:102B40008A858D83A52E542E612E702E8F2C9E2C5F
:102B5000DF86588F4C8B87C00E94C30CA22FBB8589
:102B6000AB1BA887F1E02A1708F0F0E0E32F2C85D3
:102B7000E21B21E03E1708F020E03E2F3F1BF1E072
:102B8000E31708F0F0E02F2BA42FBD85AB1BF1E07D
:102B90004A1708F0F0E04A2F421B21E0A41708F082
:102BA00020E0F22BA52FA21921E05A1708F020E00F
:102BB0005A2F5F1BF1E0A51708F0F0E02F2BA62F8E
:102BC000A419F1E06A1708F0F0E06A2F621B21E017
:102BD000A61708F020E0F22B272F2B19A1E072177F
:102BE00008F0A0E0722F7F1BF1E0271708F0F0E05B
:102BF000AF2BF82FFC1921E08F1708F020E08F2F62
:102C00008A1BA1E0F81708F0A0E02A2B9319921B69
:102C1000D91608F427C39D1529F5E81608F422C330
:102C20008E1501F5F71608F41DC37F15D9F40617A4
:102C300008F418C36017B1F4151708F413C351173B
:102C400089F4EC89E41708F40DC34E1759F4F88D94
:102C5000F31708F407C33F1729F428853A8532177C
:102C600008F400C3A8950E94B608882309F474CF1D
:102C7000588D4C894C8F5A8F0E94C408AE89BF89E9
:102C80008C9382E40E941A0938892989832F922F14
:102C900099878887805C9F4F9D8B8C8B5A8D5B8F2B
:102CA0004C8D498F8AC00E94C30CE22FBB85EB1B61
:102CB000F1E02E1708F0F0E0232FAC852A1BB1E0DD
:102CC000B88F321708F0188E322F3F1BF32F31E0E8
:102CD0002F1708F030E0A88DA32BA88F342FBD85C7
:102CE0003B1B21E0431708F020E0432FA88D4A1B2F
:102CF000A1E0341708F0A0E02A2BA52FA21931E09B
:102D00005A1708F030E05A2F521B21E0A51708F09F
:102D100020E0322BA62FA41921E06A1708F020E04A
:102D20006A2F631B31E0A61708F030E0232BA72F92
:102D3000AB1931E07A1708F030E07A2F721B21E0EE
:102D4000A71708F020E0322BA82FAC1921E08A1732
:102D500008F020E08A2F831B31E0A81708F030E04C
:102D6000232B9319921BD91608F47CC29D1521F5CB
:102D7000E81608F477C28E15F9F4F71608F472C253
:102D80007F15D1F4061708F46DC26017A9F4151762
:102D900008F468C2511781F4B98DB41708F462C2FF
:102DA0004B1751F42B8D2F1708F45CC2F21721F446
:102DB0003A853E1708F456C2A8950E94B6088823A3
:102DC00009F471CF0E94C408A885B9858D93B9878D
:102DD000A887EC89FD89AE17BF0779F782E40E94C6
:102DE0001A0909811A810F5F1F4F89819A816B81AE
:102DF0007C810E94E40C1A8309838981FE818F1BE8
:102E00002B89821708F46BCEDC2CCB2CB42C4F848E
:102E10003E853F5F3E8789819A819F838E839E8511
:102E2000AA899A1708F447CE122D2D800B2DBB844A
:102E3000FC2CCC84ED2CDD848B819C810E94F729B5
:102E400080C00E94C30CE22FEB19F1E02E1708F0AE
:102E5000F0E0232F2C19A1E0321708F0A0E0B22FE8
:102E6000BF1BFB2F31E02B1708F030E0A32B342FD2
:102E70003D1921E0431708F020E0432F4A1BA1E051
:102E8000341708F0A0E02A2BA52FA11B31E05A1718
:102E900008F030E05A2F521B21E0A51708F020E07F
:102EA000322BA62FA01B21E06A1708F020E06A2F22
:102EB000631B31E0A61708F030E0232BA72FAF19D2
:102EC00031E07A1708F030E07A2F721B21E0A71763
:102ED00008F020E0322BA82FAE1921E08A1708F065
:102EE00020E08A2F831B31E0A81708F030E0232B65
:102EF0009319921B491608F4B5C1941509F5981653
:102F000008F4B0C18915E1F4871608F4ABC178154F
:102F1000B9F4761608F4A6C1671591F4651608F49D
:102F2000A1C1561569F4541608F49CC1451541F425
:102F3000AF1608F497C1FA1519F42E1608F492C1C9
:102F4000A8950E94B608882309F47BCF0E94C40884
:102F500080C00E94C30CE22FEB19F1E02E1708F09D
:102F6000F0E0232F2C19A1E0321708F0A0E0322F57
:102F70003F1BF32F31E02F1708F030E0A32B342F45
:102F80003D1921E0431708F020E0432F4A1BA1E040
:102F9000341708F0A0E02A2BA52FA11B31E05A1707
:102FA00008F030E05A2F521B21E0A51708F020E06E
:102FB000322BA62FA01B21E06A1708F020E06A2F11
:102FC000631B31E0A61708F030E0232BA72FAF19C1
:102FD00031E07A1708F030E07A2F721B21E0A71752
:102FE00008F020E0322BA82FAE1921E08A1708F054
:102FF00020E08A2F831B31E0A81708F030E0232B54
:103000009319921B491608F42DC1941509F59816C9
:1030100008F428C18915E1F4871608F423C178154E
:10302000B9F4761608F41EC1671591F4651608F414
:1030300019C1561569F4541608F414C1451541F424
:10304000AF1608F40FC1FA1519F42E1608F40AC1C8
:10305000A8950E94B608882309F47BCF0E94C40873
:1030600080C00E94C30CE22FEB19F1E02E1708F08C
:10307000F0E0232F2C19A1E0321708F0A0E0B22FC6
:10308000BF1BFB2F31E02B1708F030E0A32B342FB0
:103090003D1921E0431708F020E0432F4A1BA1E02F
:1030A000341708F0A0E02A2BA52FA11B31E05A17F6
:1030B00008F030E05A2F521B21E0A51708F020E05D
:1030C000322BA62FA01B21E06A1708F020E06A2F00
:1030D000631B31E0A61708F030E0232BA72FAF19B0
:1030E00031E07A1708F030E07A2F721B21E0A71741
:1030F00008F020E0322BA82FAE1921E08A1708F043
:1031000020E08A2F831B31E0A81708F030E0232B42
:103110009319921B491608F4A5C0941509F5981641
:1031200008F4A0C08915E1F4871608F49BC078154F
:10313000B9F4761608F496C0671591F4651608F48C
:1031400091C0561569F4541608F48CC0451541F425
:10315000AF1608F487C0FA1519F42E1608F482C0C9
:10316000A8950E94B608882309F47BCF0E94C40862
:103170007CC00E94C30CE22FEB19F1E02E1708F07F
:10318000F0E0232F2C19A1E0321708F0A0E0322F35
:103190003F1BF32F31E02F1708F030E0A32B342F23
:1031A0003D1921E0431708F020E0432F4A1BA1E01E
:1031B000341708F0A0E02A2BA52FA11B31E05A17E5
:1031C00008F030E05A2F521B21E0A51708F020E04C
:1031D000322BA62FA01B21E06A1708F020E06A2FEF
:1031E000631B31E0A61708F030E0232BA72FAF199F
:1031F00031E07A1708F030E07A2F721B21E0A71730
:1032000008F020E0322BA82FAE1921E08A1708F031
:1032100020E08A2F831B31E0A81708F030E0232B31
:103220009319921B4916F0F09415D1F49816D0F02A
:103230008915B1F48716B0F0781591F4761690F0F0
:10324000671571F4651670F0561551F4541650F068
:10325000451531F4AF1630F0FA1511F42E1610F0B2
:10326000A89503C080E090E00CC00E94B6088823B7
:1032700009F47FCF0E94C40882E40E941A098E815B
:103280009F810E94420D6C960FB6F894DEBF0FBE70
:10329000CDBFCF91DF911F910F91FF90EF90DF9005
:1032A000CF90BF90AF909F908F907F906F905F90E6
:1032B0004F903F902F90089583E20E941A0908953D
:1032C0001F93CF93DF930E94370CEC01009731F4EA
:1032D00085E10E94700D0E945A091FC086E10E947C
:1032E000700D0E945A0910E3812F0E941A098DEB7C
:1032F00090E00E945A09899190E062E872E04AE009
:1033000050E00E94012C82E892E00E945A098AE073
:103310000E941A091F5F173339F7DF91CF911F9170
:103320000895AF92BF92CF92DF92EF92FF920F93E8
:103330001F938EE00E94700D0E945A090E94C30CD8
:10334000B901CA0142E852E02AE030E00E94222C92
:103350000E945A0980EC90E00E945A090E94C30C16
:10336000992381F4882371F4772361F4662351F45F
:10337000552341F4442331F43B3E20F43A3E09F511
:103380002136F8F083EC90E00E945A090E94C30CA9
:10339000B0E6AB2EAAEEBA2ECC24DD24EE24FF2418
:1033A00000E010E00E945E1CC90162E872E04AE0A1
:1033B00050E00E94012C0E945A0986EC90E00E9485
:1033C0005A090E94C30C992391F4882381F477232E
:1033D00071F4662361F4552351F4442341F43430ED
:1033E00030F4333009F04BC0293E08F448C083EC78
:1033F00090E00E945A090E94C30CF8EEAF2EE3E061
:10340000BE2ECC24DD24EE24FF2400E010E00E9438
:103410005E1CC90162E872E04AE050E00E94012CA3
:103420000E945A090E94C30C0E949222C90162E8BC
:1034300072E04AE050E00E94012C809182028823D1
:1034400019F08EE20E941A0980918402882319F4EF
:1034500080E30E941A0980918302882319F480E393
:103460000E941A0980918202882321F082E892E06A
:103470000E945A098CEC90E00E945A0903C08AE02D
:103480000E941A091F910F91FF90EF90DF90CF904B
:10349000BF90AF900895AF92BF92DF92EF92FF92EC
:1034A0000F931F93DF93CF930F92CDB7DEB77C01BD
:1034B0005C0110E3D12E8D2D0E941A098DEB90E056
:1034C0000E945A09850120E0F80181918F0190E066
:1034D00062E872E040E150E029830E94012C82E81A
:1034E00092E00E945A0980E20E941A0929812F5F06
:1034F000283051F78AE00E941A09D39488E090E0BE
:10350000A80EB91E9D2D9833B1F683E20E94700D6E
:103510000E945A09F701E05CFF4F808190E062E869
:1035200072E04AE050E00E94012C82E892E00E94A2
:103530005A098AE00E941A090F90CF91DF911F91DA
:103540000F91FF90EF90DF90BF90AF900895FF92A2
:103550000F931F93CF93DF93FF24A8950E94B60883
:103560008823D9F3CF2DD0E00E94C4088E010E57D6
:103570001D4FF80180830E941A09F80180818A306A
:1035800019F0FF2DF03559F4CE57DD4F188282E83F
:1035900092E0DF91CF911F910F91FF9008958D30B0
:1035A000E1F2883011F4FA94D8CFF394D6CFDF93B8
:1035B000CF930F92CDB7DEB789830E94A71A60E040
:1035C00070E0498150E00E94E42ACB010F90CF9136
:1035D000DF910895CF93DF93462FC2E8D2E090E0C9
:1035E000BE0150E00E94012CCE010E945A09DF91D9
:1035F000CF910895EF92FF920F931F93DF93CF9394
:103600000F92CDB7DEB781E490E00E945D29182FBC
:10361000092FE82EF92E83E20E94700D0E945A09AC
:103620008AE00E94D71AF701E05CFF4F8083C8014F
:10363000092F182F20E0822F6AE029830E94EA1ABE
:103640008DEB90E00E945A0980E10E94D71AF801A0
:1036500081938F0129812F5F203469F781E20E94D5
:10366000700D0E945A09C7010F90CF91DF911F91F1
:103670000F91FF90EF900895FF920F931F93DF93A8
:10368000CF93CDB7DEB729970FB6F894DEBF0FBE44
:10369000CDBF8E010F5F1F4F88E0F80111928A9510
:1036A000E9F784E20E94700D0E945A098AE00E94A4
:1036B000D71AF82E85E20E94700D0E945A0920E068
:1036C000822F6AE029870E94EA1A8DEB90E00E941F
:1036D0005A0980E10E94D71AF80181938F01298548
:1036E0002F5F283069F786E20E94700D0E945A0908
:1036F000CE0101966F2D70E042E00E94B61B81E280
:103700000E94700D0E945A0929960FB6F894DEBFE8
:103710000FBECDBFCF91DF911F910F91FF90089504
:10372000CF93DF930E94A71AC2E8D2E0CE0160E0F7
:1037300070E00E94151CFE0101900020E9F7CF0106
:1037400001978C1B9D0B23E0880F991F2A95E1F7A9
:1037500001960E94420D81E08093DB0181E20E948C
:10376000700D0E945A09DF91CF9108958F929F9218
:10377000AF92BF92CF92DF92EF92FF920F931F937F
:10378000DF93CF930F92CDB7DEB75C017B0181E46D
:1037900090E049830E945D29D82EC92E082F192F49
:1037A000F801E05CFF4F4981408340E050E020C0D9
:1037B0002815390554F4241735073CF0D501A80F16
:1037C000B11D9C9190838F5F01C010822F5F3F4F8E
:1037D00031962034310561F7C701B8010E94E40C2D
:1037E0000894E11CF11C80E48816910469F0A4019E
:1037F00088E0882E912C840E951EC601E92FFC2DA1
:1038000020E030E080E0D4CFC8010E94F7290F907B
:10381000CF91DF911F910F91FF90EF90DF90CF90AC
:10382000BF90AF909F908F9008950F931F93CF9369
:10383000DF93EB01082F192F07C00E943D1CBE012A
:1038400041E00E94B61B2896F80181918F018823E0
:10385000A1F70E948F0D8C01FC01E05CFF4F8CE012
:103860008083CE01B8010E94E40CC8010E94F729B0
:10387000DF91CF911F910F910895982F90529F350E
:1038800038F08D3011F08A3011F481E201C08FE3FD
:103890008052E82FF0E083E0EE0FFF1F8A95E1F7FA
:1038A000EE52FA4FA3EDB2E084918D93319682E00F
:1038B000AB3DB807C9F7CD0108970895A8E3B0E07C
:1038C000E4E6FCE10C94262929833A834B835C834C
:1038D0006D837E838F839887A986BA86CB86DC86A4
:1038E000ED86FE860F87188BE984FA840B851C858C
:1038F0002D853E854F85588929803A804B805C8094
:103900002DA23EA24FA258A6AD80BE80CF80D88403
:10391000211531054105510509F0A6C3AE14BF04B8
:10392000C006D10608F03FC120E0E21620E0F20612
:1039300021E0020720E0120758F43FEFE316F104FC
:103940000105110509F090F420E030E0A90117C04D
:1039500040E0E41640E0F40640E0040741E01407CC
:1039600050F420E130E040E050E009C028E030E0D1
:1039700040E050E004C028E130E040E050E0D801F1
:10398000C701022E04C0B695A795979587950A940E
:10399000D2F780539F4FDC016C9180E290E0A0E071
:1039A000B0E0821B930BA40BB50B861B9109A109F8
:1039B000B1090097A105B105A1F1082E04C0EE0CD4
:1039C000FF1C001F111F0A94D2F7A6019501082EB3
:1039D00004C0220F331F441F551F0A94D2F760E220
:1039E00070E0681B790BADA0BEA0CFA0D8A404C026
:1039F000D694C794B794A7946A95D2F7A22AB32A0B
:103A0000C42AD52A2DA03EA04FA058A404C0220C41
:103A1000331C441C551C8A95D2F72DA23EA24FA2FE
:103A200058A6380188249924A80197014070507045
:103A3000298F3A8F4B8F5C8FC601B501A40193018A
:103A40000E940429222E532E442E352E6D8F7E8FF8
:103A50008F8F98A3C601B501A40193010E94042988
:103A6000822D952DA42DB32D1C012D01C201B10174
:103A7000298D3A8D4B8D5C8D0E94E5285B016C0190
:103A80004D8D5E8D6F8D78A1DA01992788274DA124
:103A90005EA16FA178A59B0144275527822B932B0C
:103AA000A42BB52B8A159B05AC05BD05E0F4089445
:103AB00021083108410851088E0D9F1DA01FB11F1C
:103AC0008E159F05A007B10770F08A159B05AC0500
:103AD000BD0548F4089421083108410851088E0DAD
:103AE0009F1DA01FB11F9C01AD012A193B094C0964
:103AF0005D0959016A01CA01B901A40193010E943B
:103B0000042929A739A349AB5DA76D8F7E8F8F8FBD
:103B100098A3C601B501A40193010E940429A9A498
:103B2000B9A0C9A8DDA4C601B501298D3A8D4B8D78
:103B30005C8D0E94E5283B014C016D8D7E8D8F8D43
:103B400098A1AB01332722278DA19EA1AFA1B8A5D3
:103B5000A070B070282B392B4A2B5B2B261537050C
:103B600048055905C0F40894A108B108C108D10856
:103B70002E0D3F1D401F511F2E153F0540075107B9
:103B800050F0261537054805590528F40894A10872
:103B9000B108C108D1088101FF24EE24EA28FB28DE
:103BA0000C291D29A1C4E114F1040105110559F4E2
:103BB00061E070E080E090E0A80197010E94042994
:103BC00079018A0110C070E0E71670E0F70671E035
:103BD000070770E0170758F48FEFE816F1040105A6
:103BE000110509F090F420E030E0A90117C090E041
:103BF000E91690E0F90690E0090791E0190750F402
:103C000020E130E040E050E009C028E030E040E052
:103C100050E004C028E130E040E050E0D801C701A6
:103C2000022E04C0B695A795979587950A94D2F76A
:103C300080539F4FDC018C91280F311D411D511D78
:103C400080E290E0A0E0B0E0821B930BA40BB50BE8
:103C500061F4150126012E183F08400A510A81E03F
:103C6000A82EB12CC12CD12C23C1082E04C0EE0CDF
:103C7000FF1C001F111F0A94D2F715012601022E06
:103C800004C056944794379427940A94D2F7350188
:103C90004601082E04C0660C771C881C991C0A94E7
:103CA000D2F76D8E7E8E8F8E98A28DA09EA0AFA033
:103CB000B8A404C0B694A794979487942A95D2F791
:103CC000A5019401AD8CBE8CCF8CD8A0A22AB32ABA
:103CD000C42AD52AAD8EBE8ECF8ED8A22DA13EA1EC
:103CE0004FA158A504C0220F331F441F551F8A95AA
:103CF000D2F72DA33EA34FA358A7380188249924B7
:103D0000B801A7016070707049A75AA76BA77CA77C
:103D1000C201B101A40193010E940429298F39AB8A
:103D20004DA75DAB69A37AA38BA39CA3C201B1018C
:103D3000A40193010E940429A98CB9A8CDA4DDA8EF
:103D4000A98EBA8ECB8EDC8EC601B50129A53AA507
:103D50004BA55CA50E94E5285B016C0129A03AA057
:103D60004BA05CA0D101992788272D8C3E8C4F8CCD
:103D700058A0920144275527822B932BA42BB52BB7
:103D80008A159B05AC05BD0530F5298D3A8D4B8D07
:103D90005C8D2150304040405040298F3A8F4B8FEE
:103DA0005C8F8E0D9F1DA01FB11F8E159F05A00754
:103DB000B10788F08A159B05AC05BD0560F421505C
:103DC000304040405040298F3A8F4B8F5C8F8E0D92
:103DD0009F1DA01FB11FAC01BD014A195B096C09F1
:103DE0007D095A016B01CB01BA01A40193010E9424
:103DF0000429522E432E342E252E69A37AA38BA399
:103E00009CA3C601B501A40193010E940429652C5D
:103E1000742C832C922CC401B30129A53AA54BA57F
:103E20005CA50E94E5289B01AC0169A17AA18BA148
:103E30009CA16B01BB24AA248D8D9E8DAF8DB8A152
:103E4000A070B070A82AB92ACA2ADB2AA216B30623
:103E5000C406D506E0F40894610871088108910849
:103E6000AE0CBF1CC01ED11EAE14BF04C006D106CE
:103E700070F0A216B306C406D50648F4089461088B
:103E8000710881089108AE0CBF1CC01ED11E15011F
:103E90002601221A330A440A550A898D9A8DAB8D60
:103EA000BC8D6C01BB24AA24A628B728C828D92811
:103EB0003801882499246D8E7E8E8F8E98A2A80159
:103EC00097014070507029A73AA74BA75CA7C20181
:103ED000B101A40193010E940429922E832E742E15
:103EE000652E69A37AA38BA39CA3C201B1012D8D7A
:103EF0003E8D4F8D58A10E940429892D982DA72D04
:103F0000B62D898F9A8FAB8FBC8FBC01CD0129A5AF
:103F10003AA54BA55CA50E94E5283B014C0149A1AF
:103F20005AA16BA17CA1DA01992788272DA03EA078
:103F30004FA058A4920144275527822B932BA42BE2
:103F4000B52B86159705A805B90530F5298D3A8D4D
:103F50004B8D5C8D2150304040405040298F3A8F2E
:103F60004B8F5C8F8E0D9F1DA01FB11F8E159F055F
:103F7000A007B10788F086159705A805B90560F474
:103F80002150304040405040298F3A8F4B8F5C8FFA
:103F90008E0D9F1DA01FB11FAC01BD014619570911
:103FA000680979093A014B01CB01BA012D8D3E8D8B
:103FB0004F8D58A10E940429522E432E342E252EB7
:103FC00069A37AA38BA39CA3C401B3012D8D3E8D5D
:103FD0004F8D58A10E940429652C742C832C922C9F
:103FE000C401B30129A53AA54BA55CA50E94E5280B
:103FF0001B012C0169A17AA18BA19CA1AB013327E4
:1040000022278DA19EA1AFA1B8A5A070B070282BCA
:10401000392B4A2B5B2B2215330544055505C0F47B
:10402000089461087108810891082E0D3F1D401FFA
:10403000511F2E153F054007510750F0221533053B
:104040004405550528F40894610871088108910811
:10405000898D9A8DAB8DBC8D8C01FF24EE24E628D2
:10406000F7280829192943C2A216B306C406D506A3
:1040700008F42AC2203090E0390791E0490790E027
:10408000590750F42F3F31054105510509F090F4CF
:1040900066247724430119C02030A0E03A07A0E04D
:1040A0004A07A1E05A0760F490E1692E712C812C37
:1040B000912C0BC088E0682E712C812C912C05C0AE
:1040C000B8E16B2E712C812C912CDA01C901062CE0
:1040D00004C0B695A795979587950A94D2F7805313
:1040E0009F4FFC018081680E711C811C911C80E235
:1040F00090E0A0E0B0E086199709A809B90989F411
:104100002A153B054C055D0508F4E5C12DA03EA030
:104110004FA058A42E143F044006510608F0DBC1FE
:10412000D3C189A719012A0104C0220C331C441CE5
:10413000551C8A95D2F7D801C701062C04C0B69544
:10414000A795979587950A94D2F7282A392A4A2A5B
:104150005B2AA801970109A404C0220F331F441F42
:10416000551F0A94D2F729A33AA34BA35CA3860157
:104170007501062C04C016950795F794E7940A94E8
:10418000D2F7B601A50109A404C0440F551F661F4C
:10419000771F0A94D2F74D8F5E8F6F8F78A36DA132
:1041A0007EA18FA198A504C0969587957795679570
:1041B0006A94D2F73B014C018D8D9E8DAF8DB8A1D5
:1041C00086299729A829B9298D8F9E8FAF8FB8A3EB
:1041D0005201CC24DD24A20191014070507029AB22
:1041E0003AAB4BAB5CABC801B701A60195010E948D
:1041F0000429622E932E842E752E6DA77EA78FA77D
:1042000098ABC801B701A60195010E940429E62CCC
:10421000F92C082D172DE98EFA8E0B8F1C8FC801F3
:10422000B70129A93AA94BA95CA90E94E5286DA468
:104230007EA48FA498A88301FF24EE246D8C7E8C2D
:104240008F8C98A0940144275527E22AF32A042B47
:10425000152BE616F7060807190730F5298D3A8D54
:104260004B8D5C8D2150304040405040298F3A8F1B
:104270004B8F5C8FE20CF31C041D151DE214F3043C
:104280000405150588F0E616F7060807190760F417
:104290002150304040405040298F3A8F4B8F5C8FE7
:1042A000E20CF31C041D151DE61AF70A080B190B86
:1042B000C801B701A60195010E9404292DAB3EABB0
:1042C0004FAB58AF6DA77EA78FA798ABC801B701BA
:1042D000A60195010E9404296DA87EA88FA898AC1C
:1042E000C401B30129A93AA94BA95CA90E94E528F8
:1042F0009B01AC01ADA4BEA4CFA4D8A8D501992739
:104300008827AD8CBE8CCF8CD8A06FEFE62E6FEFD8
:10431000F62E012D112DAE20BF20C022D1228A29D8
:104320009B29AC29BD2982179307A407B507E0F4A0
:1043300008946108710881089108820D931DA41DDD
:10434000B51D82159305A405B50570F08217930776
:10435000A407B50748F4089461087108810891081A
:10436000820D931DA41DB51D1C012D01221A330AB7
:10437000440A550A2D8E3E8E4F8E58A2A98CBA8CB7
:10438000CB8CDC8C8501FF24EE24E628F728082955
:104390001929AFEFAA2EAFEFBA2EC12CD12CAE2027
:1043A000BF20C022D12218014424552469A07AA03C
:1043B0008BA09CA02FEF3FEF40E050E062227322E1
:1043C0008422952269A17AA18BA19CA1AC016627C8
:1043D0007727498F5A8F6B8F7C8FC601B501A40157
:1043E00093010E94E52869A37AA38BA39CA3C6012D
:1043F000B501298D3A8D4B8D5C8D0E94E5285B01BE
:104400006C01C201B101A40193010E94E5283B01A6
:104410004C01C201B101298D3A8D4B8D5C8D0E94FA
:10442000E5289B01AC01A60CB71CC81CD91C29A00F
:104430003AA04BA05CA0C201AA27BB27A80EB91EB8
:10444000CA1EDB1EA614B704C804D90420F42050E9
:1044500030404F4F5F4FC601AA27BB27820F931FE3
:10446000A41FB51F4D8C5E8C6F8C78A04816590622
:104470006A067B0618F184159505A605B705A1F512
:104480006501BB24AA2489A19AA1ABA1BCA1A070FB
:10449000B070A80EB91ECA1EDB1E8DA19EA1AFA1D1
:1044A000B8A509A404C0880F991FAA1FBB1F0A94AE
:1044B000D2F78A159B05AC05BD05B0F40894E10858
:1044C000F1080109110910C0AA24BB246501EE24DA
:1044D000FF2487010CC0AA24BB24650181E0E82EDB
:1044E000F12C012D112D03C0AA24BB246501FE016E
:1044F000719688E0DF011D928A95E9F7E98AFA8AC8
:104500000B8B1C8BAD8ABE8ACF8AD88E2E2D3A8912
:104510004B895C896A2D7E898F89988DE896E2E1C6
:104520000C944229ACE3B0E0E8E9F2E20C942629CD
:10453000F82FE92FA986BA86CB86DC86ED86FE8623
:104540000F87188BE984FA840B851C858D859E85E1
:10455000AF85B889298F3A8F4B8F5C8F298C3A8C25
:104560004B8C5C8C2DA23EA24FA258A63B018F2EF5
:104570009E2E130124010097A105B10509F00DC37A
:104580006E147F048006910608F0F7C020E0E21662
:1045900020E0F20621E0020720E0120758F43FEF86
:1045A000E316F1040105110509F090F480E090E0B4
:1045B000DC0117C040E0E41640E0F40640E00407E8
:1045C00041E0140750F480E190E0A0E0B0E009C0C1
:1045D00088E090E0A0E0B0E004C088E190E0A0E0D6
:1045E000B0E0A8019701082E04C05695479537956D
:1045F00027950A94D2F720533F4FF9012081F0E22A
:10460000AF2EB12CC12CD12CA81AB90ACA0ADB0AC8
:10461000A21AB108C108D108AD8EBE8ECF8ED8A225
:10462000A114B104C104D10499F12D8D022E04C04E
:10463000EE0CFF1C001F111F0A94D2F7022E04C0BB
:10464000660C771C881C991C0A94D2F760E270E013
:104650006A197B09298C3A8C4B8C5C8C04C056946B
:104660004794379427946A95D2F726283728482804
:104670005928498D5A8D6B8D7C8D04C0440F551F70
:10468000661F771F2A95D2F74DA35EA36FA378A765
:10469000380188249924C801B70180709070698F0F
:1046A0007A8F8B8F9C8FC201B101A40193010E946C
:1046B0000429D22EA32EC42EB52E69A37AA38BA3D0
:1046C0009CA3C201B101A40193010E9404296D2D94
:1046D0007A2D8C2D9B2D298D3A8D4B8D5C8D0E94D2
:1046E000E5285B016C0129A03AA04BA05CA0D10198
:1046F000992788272DA03EA04FA058A492014427B7
:104700005527822B932BA42BB52B8A159B05AC0523
:10471000BD0590F48E0D9F1DA01FB11F8E159F0526
:10472000A007B10748F08A159B05AC05BD0520F42C
:104730008E0D9F1DA01FB11F9C01AD012A193B09C1
:104740004C095D0959016A01CA01B901A40193012B
:104750000E940429522E232E442E352E69A37AA3BB
:104760008BA39CA3C601B501A40193010E94042957
:10477000652D722D842D932DC5C1E114F104010521
:10478000110559F461E070E080E090E0A801970124
:104790000E94042979018A0110C050E0E51650E01A
:1047A000F50651E0050750E0150758F46FEFE616DF
:1047B000F1040105110509F090F480E090E0DC01BE
:1047C00017C070E0E71670E0F70670E0070771E0C9
:1047D000170750F480E190E0A0E0B0E009C088E065
:1047E00090E0A0E0B0E004C088E190E0A0E0B0E09C
:1047F000A8019701082E04C056954795379527952F
:104800000A94D2F720533F4FF9012081820F911D66
:10481000A11DB11D50E2252E312C412C512C281AFE
:10482000390A4A0A5B0A2D8E3E8E4F8E58A22114F9
:1048300031044104510439F464015301AE18BF0836
:10484000C00AD10AEBC02D8D022E04C0EE0CFF1C55
:10485000001F111F0A94D2F713012401082E04C06F
:1048600056944794379427940A94D2F764015301DD
:10487000022E04C0AA0CBB1CCC1CDD1C0A94D2F76F
:10488000498D5A8D6B8D7C8D04C0769567955795B3
:1048900047958A95D2F7A42AB52AC62AD72AA9A26B
:1048A000BAA2CBA2DCA2698D7A8D8B8D9C8D04C0BF
:1048B000660F771F881F991F2A95D2F76DA37EA3D5
:1048C0008FA398A7380188249924D801C701A07024
:1048D000B070898F9A8FAB8FBC8FC201B101A401D8
:1048E00093010E940429D22EA32EC42EB52E69A7AF
:1048F0007AA78BA79CA7C201B101A40193010E94D2
:1049000004296D2D7A2D8C2D9B2D298D3A8D4B8D63
:104910005C8D0E94E5285B016C0129A43AA44BA49C
:104920005CA4D1019927882729A03AA04BA05CA0BC
:10493000920144275527822B932BA42BB52B8A1544
:104940009B05AC05BD0590F48E0D9F1DA01FB11FEA
:104950008E159F05A007B10748F08A159B05AC0589
:10496000BD0520F48E0D9F1DA01FB11F9C01AD0140
:104970002A193B094C095D0959016A01CA01B901AB
:10498000A40193010E940429522E232E442E352E79
:1049900069A77AA78BA79CA7C601B501A4019301BB
:1049A0000E940429652D722D842D932D298D3A8D19
:1049B0004B8D5C8D0E94E5285B016C0149A55AA5D1
:1049C0006BA57CA5DA019927882729A13AA14BA1DB
:1049D0005CA140705070822B932BA42BB52B8A15B1
:1049E0009B05AC05BD0590F48E0D9F1DA01FB11F4A
:1049F0008E159F05A007B10748F08A159B05AC05E9
:104A0000BD0520F48E0D9F1DA01FB11F1C012D019F
:104A10002A183B084C085D08620151011801442422
:104A20005524A801970140705070298F3A8F4B8F01
:104A30005C8FC601B501A20191010E940429622E7A
:104A4000932E842E752E69A37AA38BA39CA3C601F3
:104A5000B501A20191010E940429662D792D882DAE
:104A6000972D298D3A8D4B8D5C8D0E94E5285B0139
:104A70006C0149A15AA16BA17CA1DA019927882771
:104A80006DA07EA08FA098A4940144275527822B67
:104A9000932BA42BB52B8A159B05AC05BD0590F473
:104AA0008E0D9F1DA01FB11F8E159F05A007B1077A
:104AB00048F08A159B05AC05BD0520F48E0D9F1DA1
:104AC000A01FB11F9C01AD012A193B094C095D09CA
:104AD00059016A01CA01B901A20191010E94042988
:104AE000622E932E842E752E69A37AA38BA39CA38A
:104AF000C601B501A20191010E940429662D792DFC
:104B0000882D972D298D3A8D4B8D5C8D0E94E5283F
:104B10005B016C0149A15AA16BA17CA1DA01992723
:104B200088272DA13EA14FA158A540705070822B1F
:104B3000932BA42BB52B8A159B05AC05BD0590F4D2
:104B40008E0D9F1DA01FB11F8E159F05A007B107D9
:104B500048F08A159B05AC05BD0520F48E0D9F1D00
:104B6000A01FB11F8A199B09AC09BD099C01AD01A9
:104B70000D8C04C056954795379527950A94D2F722
:104B8000298B3A8B4B8B5C8B1D8A1E8A1F8A188E51
:104B90003A894B895C8960E0DEC2681679068A062C
:104BA0009B0618F48F2F9E2FD9C2803050E09507B6
:104BB00051E0A50750E0B50750F48F3F9105A105DE
:104BC000B10509F090F4AA24BB24650119C0803016
:104BD00060E0960760E0A60761E0B60760F440E198
:104BE000A42EB12CC12CD12C0BC038E0A32EB12C9B
:104BF000C12CD12C05C028E1A22EB12CC12CD12C66
:104C00009C01AD010A2C04C0569547953795279510
:104C10000A94D2F720533F4FF9012081A20EB11C14
:104C2000C11CD11C20E230E040E050E02A193B09D1
:104C30004C095D0909F047C086159705A805B90517
:104C400048F0A98CBA8CCB8CDC8CAE14BF04C006A7
:104C5000D10638F1298D3A8D4B8D5C8D2E193F0987
:104C6000400B510B681A790A8A0A9B0AA1E0EA2EC6
:104C7000F12C012D112D698D7A8D8B8D9C8D6217F4
:104C800073078407950718F0EE24FF2487011301AA
:104C900024012E183F08400A510A2DA33EA34FA31A
:104CA00058A78DA19EA1AFA1B8A5898B9A8BAB8B7C
:104CB000BC8B2D8A3E8A4F8A588E2DA13A894B890A
:104CC0005C89622D48C22DA31C012D01022E04C057
:104CD000220C331C441C551C0A94D2F7A9A6D801F7
:104CE000C70104C0B695A79597958795AA94D2F762
:104CF000282A392A4A2A5B2A2D8E3E8E4F8E58A2A8
:104D000057016801022E04C0AA0CBB1CCC1CDD1C80
:104D10000A94D2F7ADA6BEA6CFA6D8AA1301240145
:104D200009A404C056944794379427940A94D2F760
:104D300074016301022E04C0CC0CDD1CEE1CFF1CB0
:104D40000A94D2F7898D9A8DAB8DBC8D09A404C0CD
:104D5000B695A795979587950A94D2F7C82AD92A28
:104D6000EA2AFB2AC9A2DAA2EBA2FCA2E98CFA8CFD
:104D70000B8D1C8D04C0EE0CFF1C001F111F2A950B
:104D8000D2F7E9AAFAAA0BAB1CAB0D8D1E8D2F8DA5
:104D900038A13901882499242070307009AF1AAFE6
:104DA0002BAF3CAFC201B101A40193010E940429C1
:104DB000A22ED32EE42E052F6DAB7EAB8FAB98AF1A
:104DC000C201B101A40193010E9404298A2D9D2DE5
:104DD000AE2DB02F898F9A8FAB8FBC8FBC01CD01C8
:104DE00029AD3AAD4BAD5CAD0E94E5282DA93EA999
:104DF0004FA958AD8901FF24EE2429A03AA04BA069
:104E00005CA0920144275527E22AF32A042B152B94
:104E1000E616F7060807190750F5298D3A8D4B8DD0
:104E20005C8D2150304040405040298F3A8F4B8F4D
:104E30005C8F2D8C3E8C4F8C58A0E20CF31C041D13
:104E4000151DE214F3040405150588F0E616F706AF
:104E50000807190760F42150304040405040298F26
:104E60003A8F4B8F5C8FE20CF31C041D151DE61A64
:104E7000F70A080B190BC801B701A40193010E949E
:104E80000429D22EC32EB42E552E6DAB7EAB8FAB24
:104E900098AFC801B701A40193010E9404298D2D88
:104EA0009C2DAB2DB52D5C016D01C601B50129AD61
:104EB0003AAD4BAD5CAD0E94E5288B019C014DA83D
:104EC0005EA86FA878ACB2015527442789A19AA1A2
:104ED000ABA1BCA1A070B070482B592B6A2B7B2BC7
:104EE000401751076207730700F50894A108B1083D
:104EF000C108D1086D8C7E8C8F8C98A0460D571DF3
:104F0000681D791D461557056805790570F040172D
:104F100051076207730748F40894A108B108C10853
:104F2000D108460D571D681D791DDB01CA01801B84
:104F3000910BA20BB30B89A39AA3ABA3BCA3298C9F
:104F40003A8C4B8C5C8CD101992788278A299B2924
:104F5000AC29BD292FEFE22E2FEFF22E012D112DBE
:104F6000E822F9220A231B233D0188249924ADA4B9
:104F7000BEA4CFA4D8A82FEF3FEF40E050E0A2227C
:104F8000B322C422D5224DA55EA56FA578A91B0129
:104F900044245524C801B701A60195010E94E528C3
:104FA000698F7A8F8B8F9C8FC801B701A201910105
:104FB0000E94E5287B018C01C401B301A601950183
:104FC0000E94E5285B016C01C401B301A2019101BB
:104FD0000E94E5289B01AC01EA0CFB1C0C1D1D1D69
:104FE000298C3A8C4B8C5C8CC201AA27BB27E80E1B
:104FF000F91E0A1F1B1FEA14FB040C051D0520F4F3
:10500000205030404F4F5F4FC801AA27BB27820F67
:10501000931FA41FB51F8701FF24EE24298D3A8D0D
:105020004B8D5C8D40705070E20EF31E041F151FF7
:1050300049A05AA06BA07CA0481659066A067B06B8
:1050400070F084159505A605B70599F569A87AA8A5
:105050008BA89CA86E147F048006910650F5A801C9
:1050600097018DA49EA4AFA4B8A8281939094A09AC
:105070005B095C016D012D8C3E8C4F8C58A0A218F1
:10508000B308C408D50881E090E0A0E0B0E0E216E3
:10509000F3060407150718F080E090E0DC01250115
:1050A0003601481A590A6A0A7B0AD301C2017901FA
:1050B0008A0169A87AA88BA89CA86E187F08800A24
:1050C000910A9401830149A15AA16BA17CA1481BBB
:1050D000590B6A0B7B0B81E090E0A0E0B0E089A85F
:1050E0009AA8ABA8BCA880169106A206B30618F031
:1050F00080E090E0DC01481B590B6A0B7B0B5A01E6
:105100006B0109A404C0AA0CBB1CCC1CDD1C0A94B6
:10511000D2F70DA004C036952795179507950A94E8
:10512000D2F7A02AB12AC22AD32AA98ABA8ACB8A5C
:10513000DC8ACB01BA010DA004C0969587957795BE
:1051400067950A94D2F76D8B7E8B8F8B988F2A2D63
:105150003A894B895C897E898F89988DEC96E2E14A
:105160000C944229991B79E004C0991F961708F006
:10517000961B881F7A95C9F780950895AA1BBB1BBB
:1051800051E107C0AA1FBB1FA617B70710F0A61B47
:10519000B70B881F991F5A95A9F780959095BC0168
:1051A000CD01089597FB092E07260AD077FD04D07C
:1051B000E5DF06D000201AF4709561957F4F0895C1
:1051C000F6F7909581959F4F0895629FD001739F48
:1051D000F001829FE00DF11D649FE00DF11D929F93
:1051E000F00D839FF00D749FF00D659FF00D9927D2
:1051F000729FB00DE11DF91F639FB00DE11DF91FF6
:10520000BD01CF0111240895A1E21A2EAA1BBB1BD8
:10521000FD010DC0AA1FBB1FEE1FFF1FA217B30782
:10522000E407F50720F0A21BB30BE40BF50B661F98
:10523000771F881F991F1A9469F76095709580955C
:1052400090959B01AC01BD01CF0108952F923F9233
:105250004F925F926F927F928F929F92AF92BF9286
:10526000CF92DF92EF92FF920F931F93CF93DF9332
:10527000CDB7DEB7CA1BDB0B0FB6F894DEBF0FBE8F
:10528000CDBF09942A88398848885F846E847D84DC
:105290008C849B84AA84B984C884DF80EE80FD80DE
:1052A0000C811B81AA81B981CE0FD11D0FB6F89454
:1052B000DEBF0FBECDBFED010895CF93DF938230E7
:1052C000910510F482E090E0E091DD02F091DE02C1
:1052D00040E050E020E030E026C060817181681736
:1052E0007907E0F06817790781F4828193812115AD
:1052F000310531F0D90113969C938E9312972BC0F0
:105300009093DE028093DD0226C04115510519F00D
:105310006417750718F4AB01E901DF019F01728181
:105320006381E72FF62F3097C1F64115510501F142
:10533000481B590B4430510580F412968D919C9175
:105340001397209719F09B838A8304C09093DE0201
:105350008093DD02FD01329646C0FD01E40FF51F8A
:10536000819391934250504011965C934E933BC071
:105370002091DB023091DC022115310541F42091AE
:10538000D2013091D3013093DC022093DB022091D3
:10539000D4013091D5012115310541F42DB73EB727
:1053A0004091D0015091D101241B350BE091DB02DB
:1053B000F091DC02E217F307A0F42E1B3F0B281735
:1053C000390778F0AC014E5F5F4F2417350748F07E
:1053D0004E0F5F1F5093DC024093DB028193919349
:1053E00002C0E0E0F0E0CF01DF91CF910895CF93CC
:1053F000DF93009709F491C0FC0132971382128267
:105400006091DD027091DE026115710581F42081E9
:105410003181280F391F8091DB029091DC028217C5
:10542000930799F5F093DC02E093DB0276C0DB0191
:1054300080E090E002C0CD01D901AE17BF0748F46B
:1054400012962D913C91139721153105A1F7CD01AD
:1054500021C0B383A283EF01499159919E01240F8A
:10546000351FA217B30779F42D913C911197240FA2
:10547000351F2E5F3F4F3183208312962D913C9133
:10548000139733832283009729F4F093DE02E0938D
:10549000DD0243C0DC011396FC93EE9312974D910D
:1054A0005D91A40FB51FEA17FB0769F420813181D4
:1054B000240F351F2E5F3F4FEC0139832883228153
:1054C00033813B832A83E0E0F0E002C0FB01BC01B2
:1054D000DB0112968D919C9113970097B9F79B0170
:1054E0002E5F3F4F8D919C911197820F931F40919A
:1054F000DB025091DC024817590779F4309729F400
:105500001092DE021092DD0202C01382128222503B
:1055100030403093DC022093DB02DF91CF9108957D
:10552000A0E0B0E0E6E9FAE20C942E29EC016881F3
:1055300079818A819B81611571058105910521F42D
:1055400064E279ED8BE597E02DE133EF41E050E047
:105550000E94692C79018A0127EA31E440E050E099
:105560000E94E5285B016C01C801B7012CEE34EF05
:105570004FEF5FEF0E94E5286A0D7B1D8C1D9D1D7E
:1055800097FF04C0615070408040904868837983E1
:105590008A839B837F77CB01CDB7DEB7EAE00C949B
:1055A0004A290E94902A089586ED91E00E94902A4F
:1055B0000895A0E0B0E08093D6019093D701A09326
:1055C000D801B093D90108952F923F924F925F92E4
:1055D0006F927F929F92AF92BF92CF92DF92EF92A3
:1055E000FF920F931F93CF93DF933B01EA01611565
:1055F000710519F0FB0180839183209739F09E019A
:10560000225030402332310508F0D5C0C82ED92EA3
:10561000F60111916F017F01812F90E00E94F22B22
:105620000097B1F71D3231F4F60111917F019924F1
:10563000939406C01B3219F4F60111917F0199244D
:10564000209719F0C031D105D1F4103389F4F70156
:105650008081883711F0883559F4F701118182E093
:1056600090E0E80EF91E92E0992AC0E1D0E007C070
:10567000209729F41033B1F0CAE0D0E02BC0CA3033
:10568000D10541F1C031D10521F0C830D105A9F4CF
:1056900009C02FEFA22E2FEFB22E2FEFC22E2FE038
:1056A000D22E20C0C8E0D0E09FEFA92E9FEFB92EE8
:1056B0009FEFC92E9FE1D92E15C09E01442737FDCB
:1056C0004095542F6FEF7FEFCB010E9404295901C1
:1056D0006A0108C089E9A82E89E9B82E89E9C82E8F
:1056E00089E1D82E60E020E030E0A9011E014424C9
:1056F00037FC4094542C012F00530A3060F0812F66
:1057000081548A3110F4075006C0812F81568A31A6
:1057100050F5012F0755802F90E08C179D071CF541
:105720006F3FE9F0A216B306C406D506A8F0CA0179
:10573000B901A20191010E94E5289B01AC01802FD3
:1057400090E0A0E0B0E0280F391F4A1F5B1F281728
:1057500039074A075B0710F46FEF01C061E0F701FA
:1057600011917F01C8CF6114710481F0662339F073
:105770000894E108F108F301F182E08207C091FE8C
:1057800005C0C7010297F3019183808390FE07C093
:1057900050954095309521953F4F4F4F5F4F67FF94
:1057A0000DC082E290E09093E0028093DF022FEF41
:1057B0003FEFA90103C020E030E0A901B901CA010F
:1057C000DF91CF911F910F91FF90EF90DF90CF90DD
:1057D000BF90AF909F907F906F905F904F903F9061
:1057E0002F900895911162C0803219F08950855030
:1057F000D0F70895FB01DC0105900D920020E1F740
:105800000895FB019F01E8944230C4F04532B4F49E
:105810004A3029F497FB1EF4909581959F4F642F91
:1058200077270E94BE28805D8A330CF0895D8193C2
:10583000CB010097A1F716F45DE251931082C901E4
:105840000C94592CFA01CF93FF93EF93223044F13B
:10585000253234F5C22FE894CA3049F497FB3EF460
:1058600090958095709561957F4F8F4F9F4F2C2F0E
:10587000332744275527FF93EF930E940429EF9184
:10588000FF91605D6A330CF0695D6193B901CA01F3
:10589000605070408040904051F716F4CDE2C193C3
:1058A00010828F919F91CF910C94592C9927882722
:1058B0000895DC01FC01672F71917723E1F732979E
:1058C00004C07C916D9370836291AE17BF07C8F3DB
:1058D000089597FB092E05260ED057FD04D094DCC1
:1058E0000AD0001C38F450954095309521953F4FD3
:1058F0004F4F5F4F0895F6F790958095709561959D
:0C5900007F4F8F4F9F4F0895F894FFCF0A
:10590C00202800290081422418182442810000001C
:10591C000000000000000000000000000081422494
:10592C001818244281814224181824428100000056
:10593C000000000000000000000000000081422474
:10594C0018182442810101500FC40E2E0FA00F080D
:10595C000F6A0FE60E020408101F3F7DFA3A200072
:10596C006D7300202800206D696E290073290A00D0
:10597C0000010202030303030404040404040404EA
:10598C0005050505050505050505050505050505BB
:10599C00060606060606060606060606060606069B
:1059AC00060606060606060606060606060606068B
:1059BC00070707070707070707070707070707076B
:1059CC00070707070707070707070707070707075B
:1059DC00070707070707070707070707070707074B
:1059EC00070707070707070707070707070707073B
:1059FC00080808080808080808080808080808081B
:105A0C00080808080808080808080808080808080A
:105A1C0008080808080808080808080808080808FA
:105A2C0008080808080808080808080808080808EA
:105A3C0008080808080808080808080808080808DA
:105A4C0008080808080808080808080808080808CA
:105A5C0008080808080808080808080808080808BA
:105A6C0008080808080808080808080808080808AA
:0A5A7C002000E1020000010000001C
:00000001FF
